:100000000C942A000C9445000C9445000C94450077
:100010000C9445000C9445000C9445000C9445004C
:100020000C9445000C9445000C9445000C9445003C
:100030000C9445000C9445000C9445000C9445002C
:100040000C9445000C9445000C9445000C9445001C
:100050000C94450011241FBECFE5D8E0DEBFCDBF14
:1000600010E0A0E6B0E0E4EFF2E002C005900D92EF
:10007000AA36B107D9F710E0AAE6B0E001C01D9298
:10008000A637B107E1F70C9421010C94000084E835
:1000900086B908951CBE13BC8BE783BF8AE785BD74
:1000A000089510BC89E189B982E08BB980E98AB9E9
:1000B00086E880BD0895877087B9369A3699FECF55
:1000C00084B195B10895882339F083BD959A66234C
:1000D00039F06CBF969A089513BC95986623C9F7BA
:1000E0001CBE9698089590916E009A3089F09B30CE
:1000F00038F0943169F0953141F19B3099F10895D0
:100100009923C9F48035D9F781E080936E00089572
:100110008A3344F48295807F809375009F5F90932B
:100120006E00089587508295807F809375009F5F51
:1001300090936E000895913011F7883521F189353B
:10014000D9F484E180936E0008958A33C4F48F70EB
:1001500090917500892B8093750080936F001092A9
:100160006E0008958A336CF48F7090917500892B1E
:10017000809375008093720010926E0008958750EE
:10018000E6CF8750F1CF8AE080936E000895CF9339
:10019000DF93CFEFD0E00E9449010E94730080916D
:1001A00072009927880F991F805091409093740096
:1001B0008093730020916F003327220F331F20504C
:1001C000314030936B0020936A004396879720F468
:1001D00010927400109273002D5E3F4F273231054C
:1001E00020F410926B0010926A008091730090913D
:1001F000740020916A0030916B00AC01420F531FD4
:100200005093710040937000281B390B30936D00A0
:1002100020936C004F3F510529F024F0D0937100DA
:10022000C09370002F3F310529F024F0D0936D006A
:10023000C0936C0060916C00809170000E9463001C
:10024000AACFCFE5D8E0DEBFCDBF83E08ABB8BE08D
:1002500087BB14BA10E811BB0E9447000E944A00F5
:100260008FEC90E00E94400180E690E00E946A01DD
:100270001093720010936F000E94C7000C947901D4
:10028000292F332720BD89B988E18AB98EE880BD3E
:1002900008955F9BFECF8CB1992708955D9BFECF9B
:1002A0008CB908951F93282F982F92959F70892FAE
:1002B000805D8A3308F0895F922F9F70192F105D3F
:1002C0001A3308F0195F0E944E01812F0E944E01DF
:1002D0001F910895CF93DF93EC018881882331F03B
:1002E0000E944E01219688818823D1F7DF91CF911A
:0402F0000895FFCF9F
:0A02F40052454144592E0A0D000046
:00000001FF
